:020000040000FA
:1000000083160313CF308500C1308600813087000E
:100010008312031300309F008316031788008900A2
:10002000831203170730870088008316031370308C
:100030008F00F5309000243098000330990083122F
:10004000031390309800831603133030920083120C
:1000500003130C30920018309B0020309D000130BB
:10006000900000308E008F000C10831603130C14C8
:1000700083120313003085000130860001308700B1
:100080000A27B30114246630840008302224331177
:10009000851B672850306E06031D672833156F08CF
:1000A000A00083136E3084000C30A100840A840AFF
:1000B0000008840384038000840AA10B56282030A2
:1000C000FA00FB0066308400083044246D2850306C
:1000D0006C06031D73286D08A0003130A0020830A3
:1000E0002002031C77282030EC00ED008C285030D3
:1000F000EC0031302007ED004C3084002008222431
:100100004C08E6004D08E7004E08E8004F08E900FB
:100110005008EA005108EB005A260030B9001030B0
:10012000BA00BC2665261230B9001030BA00BC26D1
:1001300070262330B9001030BA00BC267B2633303D
:10014000B9001030BA00BC26C9235030A000502698
:100150007522B4300F02031CA928A00BA728331066
:100160008A26C9237522AB229224FF3A031DB228A6
:10017000851B33117522AB229224FF3A0319B8284C
:10018000FF3AB800331DCB280E303806031DAF28C8
:100190000A128A156B28B808031DE5283030680656
:1001A000031DE22837306606031DDA28363067065D
:1001B0000319F928E7032F306706031DE2283930B9
:1001C000E700E6033030E8004D2901303806031916
:1001D000ED2815303806031D102937306606031D3B
:1001E000002936306706031D002930306806031DDC
:1001F00000293930E6003530E7003030E8000F29BB
:10020000E8032F306806031D0F293930E800E703A3
:100210002F306706031D0F293930E700E6034D290B
:10022000023038060319182914303806031D3729FF
:1002300039306606031D272935306706031D272937
:100240003730E6003630E7003030E8003629E80A7B
:100250003A306806031D36293030E800E70A3A30A4
:100260006706031D36293030E700E60A4D290330C2
:100270003806031D50293030E80039306606031D6A
:1002800045293530670603192029E70A3A30670601
:10029000031D4D293030E700E60AB31C1424AF28B3
:1002A00004303806031D58290030A00031308F2952
:1002B00005303806031D60290130A00032308F2937
:1002C00006303806031D68290230A00033308F291C
:1002D00007303806031D70290330A00034308F2901
:1002E00008303806031D78290430A00035308F29E6
:1002F00009303806031D80290530A00036308F29CB
:100300000A303806031D88290630A00037308F29AF
:100310000B303806031DA3290730A0003830ED004C
:100320005030EC004C308400200822244C08E600B9
:100330004D08E7004E08E8004F08E9005008EA00C1
:100340005108EB00AF280C303806031DB2296A08AB
:100350006F24A0000C39EA00200A03396A047B24C8
:10036000EA00AF280D303806031DC0296B086F2442
:10037000A0000430A0070F3020057B24EB00AF283D
:100380000E303806031DC529EF2910303806031931
:10039000CD2913303806031DD92950306C06031DB2
:1003A000D72931306D060319D7292E30EA290B30B1
:1003B000ED29113038060319E12912303806031DE2
:1003C000AF2850306C06031DEC2938306D06031938
:1003D000EC292C306D02ED290430B800CB28331401
:1003E000B8018A26AB2270264530B9001030BA0019
:1003F000BC267B263808A000A00AA00B032A503098
:10040000B9001030322AA00B092A5A30B900103036
:10041000322AA00B0F2A6A30B9001030322AA00B02
:10042000152A7F30B9001030322AA00B1B2A8F30DA
:10043000B9001030322AA00B212AA130B9001030A7
:10044000322AA00B272AB030B9001030322AA00B74
:100450002D2AC030B9001030322AA00BF029D0303C
:10046000B9001030BA00BC268824A0000F30200646
:10047000031D3B2AAF2814302006031D452AB80A65
:10048000093038060319B800F12915302006031D7C
:10049000502AB803FF30380608300319B800F12994
:1004A0000E302006031D342A0A128A153808A000CF
:1004B00003190028A00303196B28A00303193C2982
:1004C000A00303198F2AA0030319402BA0030319CB
:1004D000452CA0030319A12CA0030319E82CA003A9
:1004E0000319882D0A128A11F029702566084D25F6
:1004F00067084D2568084D2569084D256A084D2572
:100500006B084D250D304D255525003A031DA42AB5
:100510003F08C8005525003A031DA42A3F08C9001A
:100520005525003A031DA42A3F08CA005525003A64
:10053000031DA42A3F08CB005525003A031DA42A19
:100540000D303F06031908004330C8003030C900A1
:10055000CA00CB00A32A0030A0266C08EF266D0845
:10056000EF262030EF266608EF266708EF262E30AC
:10057000EF266808EF264D30EF264830EF267A3018
:10058000EF262030EF264808A2016F2401393130D0
:10059000031DCC2AA20A2030EF26220BD42A3030A9
:1005A000490620300319D52A4908EF264A08EF26C4
:1005B0006430EF264230EF262030EF2648086F24C3
:1005C000A200A218F32A2219F92AA219ED2A023050
:1005D000EF265330EF265430FE2A0330EF264D30FD
:1005E000EF264E30FE2A4F30EF265630EF264630AB
:1005F000FE2A2D30EF262D30EF262D30EF2640300D
:10060000A0268313523084001430A2000008EF2685
:10061000840AA20B062B1430A0266A086F24033923
:10062000A200A20AA20B202B7330EF262E30EF2659
:100630007730EF266930EF266430EF266530472BA0
:10064000A20B2E2B7730EF266930EF266430EF2691
:100650006530EF262030EF262030472BA20B3C2BB5
:100660006D30EF266930EF266430EF266430EF26D8
:100670006C30EF266530472B6E30EF266130EF2669
:100680007230EF267230EF266F30EF267730EF268C
:100690002030EF266B086F24A200A219552B613081
:1006A000EF267530EF2674305A2B6D30EF266F3001
:1006B000EF266E30EF266F30EF262030EF266D30BC
:1006C000EF267530EF267430EF266530EF262D309B
:1006D000EF266F30EF262219712B6E30EF26203077
:1006E000742B6630EF266630EF267B26331D872B72
:1006F0007030EF267230EF266F30EF266730EF262E
:100700007230EF266130EF266D30EF26A42BB31840
:10071000962B6E30EF266F30EF267230EF266D305D
:10072000EF266130EF266C30EF26A42B7330EF26D6
:100730007030EF266530EF266330EF266930EF2604
:100740006130EF266C30EF262030EF266B086F24E7
:10075000A200A21CAF2B3130EF269230B22B963084
:10076000221C4830D0266B30EF264830EF267A30F6
:10077000EF262030EF264C30EF2669086F240F3922
:10078000A2000A3022020030031806302207D026C9
:10079000080037306602031CF92B3A306602031852
:1007A000F92B30306702031CF92B3A30670203182B
:1007B000F92B30306802031CF92B3A306802031819
:1007C000F92B37306602031DE92B36306702031C14
:1007D000F92B39306602031D002C363067020318EE
:1007E000F92B35306702031D002C303068020319E5
:1007F000002C3730E6003630E7003030E8001424B3
:1008000069086F240F397B24E9006A086F240339D3
:100810007B24EA006B086F240C39EB007C08033959
:100820006B047B24EB0008002030EC00ED00831308
:10083000523084001430A40020308000840AA40BBD
:100840001D2C0800A2000310220DA200A300A20D7F
:10085000220DA200A307220D2307A2008312031773
:100860008D008312031383131A30A200831603171B
:100870000C14831203170C0880008D0A840A83125B
:100880000313A20B362C0800A2000310220DA200B5
:10089000A300A20D220DA200A307220D2307A20090
:1008A000831203178D008312031383131A30A200DF
:1008B0000008831203178C00831603170C1555309C
:1008C0008D00AA308D008C148C18642C83120317B1
:1008D0008D0A840A83120313A20B582C0800A4006B
:1008E0003030A4020A302402031C782C0730A40202
:1008F0000F3024050800A4000F30A4053030A407F1
:100900003A302402031C862C0730A4072408080070
:100910009224FF3A031D882C9224FF3A03198C2C51
:10092000FF3A08008312031386160630A200A20BBA
:10093000972C050886120F39BE000C303E18A92CE2
:100940000D30BE18A92C0E303E19A92C0F30BE1D3B
:10095000B42CA2002430A400DB30A300A30BAE2CE7
:10096000A40BAE2C22084C2D3318D22C0626003AAC
:10097000031DD22C12304406031DD22C3430450600
:10098000031DD22C46084707FF3A031DD22CF03036
:100990004605031DD22C0E304602003003180230EB
:1009A00046074C2D86150630A200A20BD52CF03040
:1009B000B4050F300505B4048611B5103510133099
:1009C0003405013A031DE72CB51235163614361CD2
:1009D000F42C03303405033A031DF42CFC30B50528
:1009E000350E0339B504361023303405023A031DA1
:1009F000FC2CB5163512B614B61C092D033034057F
:100A0000033A031D092DFC30B505350E0339B50435
:100A1000B610CF30B405340E3039B404B5113511E9
:100A20004C303405043A031D182DB513351736150F
:100A3000361D252D0C3034050C3A031D252DF330C1
:100A4000B505350E0C39B50436118C303405083A2D
:100A5000031D2D2DB5173513B615B61D3A2D0C30C7
:100A600034050C3A031D3A2DF330B505350E0C391B
:100A7000B504B6113F30B405340EC039B404123099
:100A800035184C2D1330B5184C2D143035194C2D0C
:100A90001530B5194C2DFF30080083160313981C30
:100AA0004F2D83120313990008000030BF008C1AE9
:100AB0005F2D5A2D5B2DBF0B572D03306F2D18194D
:100AC000672D98186A2D1A08BF0000306F2D1A087C
:100AD00001306F2D181200000000181602300800B7
:100AE0001A081A08181200000000181608008F25AE
:100AF0002030A200C70DC60DC50DC40D0318822DF0
:100B0000BD25832DA625A20B7A2DD4254F30A30019
:100B1000DE30A200A20B8A2DA30B8A2D08002C30F8
:100B20009D001630A5007D30A400A40B952DA50BCB
:100B3000952D20309D00FD3087050B30A500BC3081
:100B4000A400A40BA12DA50BA12D08002C309D0005
:100B50000230A5005030A400A40BAC2DA50BAC2D89
:100B600020309D00FD3087050530A5000830A40029
:100B7000A40BB82DA50BB82D08002C309D00023019
:100B8000A5005030A400A40BC32DA50BC32D20300D
:100B90009D00FD3087050230A5005030A400A40B55
:100BA000CF2DA50BCF2D08002C309D000230A500C5
:100BB0005030A400A40BDA2DA50BDA2D20309D00B7
:100BC000FD3087050800A4000310A40DA40D24081F
:100BD0009F3EA4001230A5000318A50A02260A129F
:100BE0008A11C400FF250A128A11C500FF250A12C6
:100BF0008A11C600FF250A128A11C7000800A40A3C
:100C00000319A50A25088A00240882000130071864
:100C10004F2E50260718122E56300F02031C0A2E94
:100C200006304F2E3A305026071C1C2E32300F0251
:100C3000031C142E07304F2E1D300F020330031CEF
:100C40004F2E2030A500502607182C2E16300F02EC
:100C5000031C242E08304F2E5026071C352E16302C
:100C60000F02031C2D2E09304F2E08300F02C70D26
:100C7000C60DC50DC40DA50B232E50260718462EF4
:100C800016300F02031C3E2E0A304F2E5026053020
:100C9000071C4F2E0E300F02031C472E0030080099
:100CA00000308E008F000C10831603130C14831277
:100CB000031308000030A0261430A2002030EF26D5
:100CC000A20B5E2E0030A02608004030A026143073
:100CD000A2002030EF26A20B692E4030A02608008B
:100CE0001430A0261430A2002030EF26A20B742E60
:100CF0001430A02608005430A0261430A200203062
:100D0000EF26A20B7F2E5430A026080018308B2E21
:100D100034308B2E3030A200C3308705070805120F
:100D20006127C33087052208870405126127053033
:100D3000A3000A30A200A20B9B2EA30B9B2E08003F
:100D4000A400A500A50CA50C3C30A505A516C33034
:100D500087052508870405126127A40DA40D3C30E2
:100D6000A405C330870524088704051261271830BD
:100D7000A500A50BB92E0800CC260A128A11003A4C
:100D80000319CB2EFF3A0319CB2EFF3AEF26B90AEF
:100D90000319BA0ABC2E08003A088A0039088200F2
:100DA000A200F039A3000310A30CA30CA30CA30C06
:100DB0003030A3073A302302031CE02E0730A3078C
:100DC0000F30A2053030A2073A302202031CEA2E6F
:100DD0000730A2072308EF262208EF260800A40008
:100DE000A500A50CA50C3C30A505C330870525083A
:100DF000870405166127A40DA40D3C30A405C3305B
:100E0000870524088704051661271830A500A50B5F
:100E1000072F08006030A3009F30A200A20B0E2F06
:100E2000A30B0E2F6400C33087050C308704051216
:100E300061270A30A300D230A200A20B1D2FA30B02
:100E40001D2FC33087050C308704051261273D3004
:100E5000A200A20B292FC33087050C30870405128E
:100E600061273D30A200A20B332FC33087058715C1
:100E7000051261273D30A200A20B3C2FC33087052D
:100E8000871505126127C33087058716051261276C
:100E90003D30A200A20B4A2F86268A26C330870542
:100EA000071605126127C330870505126127183020
:100EB000A200A20B592FDF30B9001230BA00BC26B5
:0A0EC00008008516000085120800E6
:1010000050306C060030031D072831306D02A000FF
:101010000A128A117026E030B9001030BA00BC26DE
:101020007B26E830B9001030BA00BC2688260A12A8
:101030008A15083020060A3003191F28200AA1004B
:10104000543021070A128A11A0260A128A11882414
:101050000A128A15A1000F302106031D32280A1238
:101060008A11F12914302106031D3C28A00A0930F9
:1010700020060319A000192815302106031D472852
:10108000A003FF30200608300319A00019280E30F5
:101090002106031D25280830200603196428660848
:1010A000CC006708CD006808CE006908CF006A0848
:1010B000D0006B08D1005030EC0031302007ED003B
:1010C0004C308400200867286630840008300A12FB
:1010D0008A114424AF28A030840008300A128A11F3
:1010E00022240A128A15331D81280A128A117026B9
:1010F0001C30B9001130BA00BC267B260A128A15B2
:1011000096280A128A116526F930B9001030BA0003
:10111000BC267B260730B9001130BA00BC268826D1
:10112000A0010A128A1170260A128A158313A830A8
:1011300084000730A10050300006031DA9280A12C0
:101140008A110008EF26840A0008EF260A128A1581
:10115000B228840A0A128A112A30EF262A30EF2692
:101160000A128A15840AA1030319BD2820300A1225
:101170008A11EF260A128A159B283319D0280830C5
:1011800020060A300319CA28093020061030031936
:10119000CA28200AA100543021070A128A11A02669
:1011A0000A128A1188240A128A15A1000F3021061A
:1011B000031DDF280A128A11331DF129AF283319C4
:1011C000D02814302106031DEB28A00A0A3020067F
:1011D0000319A000BF2815302106031DF628A0031F
:1011E000FF30200609300319A000BF280E30210669
:1011F000031DD02808302002031C012903192A29C5
:1012000035298313A83084000730A1005030000630
:10121000031911295030800031302007840A8000E2
:101220009128840A840AA10B06298313A83084001C
:101230000C30A100840A840A00088403840380001F
:10124000840AA10B1A295030800031302007840A0B
:10125000800091288313A83084000E30A100203034
:101260008000840AA10B30299028A0308400083027
:101270000A128A114424AF2883136630A000A030DC
:10128000A1000630A200200884000008A300210865
:10129000840023088000A00AA10AA20B432983131B
:1012A0005230A000A630A1001430A2002008840013
:1012B0000008A3002108840023088000A00AA10AD6
:1012C000A20B56290A128A1165262C30B90011305A
:1012D000BA00BC2670268313A63084001430A00008
:1012E00000080A128A11EF260A128A15840AA00B36
:1012F0007029BB010A128A117B2688260A128A15D8
:101300007D2214303B070A128A11A0260A128A1580
:1013100085223D080A128A11EF263C087F39F83EE3
:10132000A0000030031C6030A007BC1BA017543085
:10133000A0260A128A156D226D226D226D226D2261
:101340006D226D226D2200300A128A11EF260A12D8
:101350008A156D2201300A128A11EF260A128A15A7
:101360006D226D226D226D226D226D226D226D2205
:101370006D2214303B070A128A11A0260A128A1124
:1013800088240A128A15A1000F302106031DCB29DB
:101390000A128A11F1290C302106031DD4297D225D
:1013A0008030BC0685227E2915302106031DE129E7
:1013B000BC0A3C087F39603A031DF0298030BC0527
:1013C000F02914302106031DF229BC033C087F39A3
:1013D0007F3A031DF0293C088039803A5F38BC0011
:1013E00085227E2912302106031DFE29BB0A1430F6
:1013F0003B06031D7E290030BB007E2913302106E9
:10140000031D0A2ABB03FF303B06031D7E29133050
:10141000BB007E290E302106031DBE290A128A1147
:101420007B263F30B9001130BA00BC260A128A155B
:1014300050306C060030031D1F2A31306D02A000B1
:10144000553020070A128A11A0260A128A11882410
:101450000A128A15A1000F30210603197A291430C7
:101460002106031D392AA00A083020060319A0000E
:10147000202A15302106031D442AA003FF30200630
:1014800007300319A000202A0E302106031D252A4B
:10149000A030840020080A128A1144240A128A15F6
:1014A00050306C060030031D692A4C308400313006
:1014B0006D020A128A1122244C08E6004D08E7004A
:1014C0004E08E8004F08E9005008EA005108EB0018
:1014D000AF280A128A111424AF282008203E0A12CD
:1014E0008A11EF260A128A15A00A20087F39603A6D
:1014F000031D7C2A8030A00508008313A6303B071B
:1015000084000008E03EBC0008003C08203EBD000E
:101510008313A6303B0784003D0880000800A0012B
:101520000A128A1170264930B9001130BA00BC265F
:101530000A128A117B260A128A150030B90013306C
:10154000BA002008B9070318BA0A3323A1003323CD
:10155000BA002108B9000A128A11BC260A128A159B
:1015600033230A128A1188240A128A15A1000F3027
:101570002106031DBE2A0A128A11F1291430210600
:10158000031DC92A1E30200603198F2A0230A00726
:10159000982A15302106031DD62AA008031DD32A38
:1015A0001E30A000982A0230A002982A0E30210690
:1015B000031DB12AA001A1011E23A1080319EB2AD2
:1015C000831603133730A0003630A1003030A2005C
:1015D000831203130E2B332383160313A00033232C
:1015E00083160313A100332383160313A20083126F
:1015F00003138313A63084003323A200A208031927
:101600000E2BFF30220603190D2BBA3004060319E6
:10161000FC2A22088000840AFC2AA10AA030840047
:1016200020080A128A1144240A128A15A00A0830D6
:101630002006031DDC2A0A128A114228831603138E
:101640003330A3003130A4003030A5008313A6301E
:101650008400143083120313A20020308000840A17
:10166000A20B2E2B0800831203133C230A128A15A7
:10167000B90A0319BA0A08003A088A003908820030
:10168000A0010A128A1165260A128A150030B900D3
:101690001330BA002008B9070318BA0A3323A1008F
:1016A0003323BA002108B9000A128A11BC260A1293
:1016B0008A1533233908C0003A08C1003908C2002E
:1016C0003A08C3000A128A1170260A128A154208C3
:1016D000B9004308BA000A128A1533230A128A1184
:1016E000EF260A128A1533230A128A11EF262E30AA
:1016F000EF260A128A1533230A128A11EF262030A8
:10170000EF26BC265A265730B9001130BA00BC2645
:101710007B260A128A1188240A128A15A1000F302A
:101720002106031D962B0A128A11F1291230210677
:10173000031DA12B1E3020060319402B0230A007E9
:10174000412B13302106031DAE2BA008031DAB2B2C
:101750001E30A000412B0230A002412B1430210684
:10176000031DBE2B4208B9004308BA003323FF3AD9
:101770000319622BFF3A031DB62B5E2B1530210691
:10178000031DE02B42084006031DCA2B43084106F7
:101790000319622B4208B9004308BA00B903FF30AD
:1017A00039060319BA03B903FF3039060319BA031E
:1017B0003C230A128A15003A031DD32B33235E2BD8
:1017C0000E302106031D892B0A128A117B263F3019
:1017D000B9001130BA00BC26BC0188260A128A1151
:1017E00055303C07A0260A128A1188240A128A154D
:1017F000A1000F30210603193F2C14302106031DD0
:10180000072CBC0A08303C060319BC00EE2B15302F
:101810002106031D122CBC03FF303C0607300319C0
:10182000BC00EE2B0E302106031DF32B4208B9003D
:101830004308BA001E23332383160313A000332367
:1018400083160313A100332383160313A20083130B
:10185000A63084003323FF3A0319372CFF3A0319CB
:10186000372C8000840ABA300402031C2A2C83120D
:101870000313A03084003C080A128A1144240A127F
:101880008A118A260A128A15622B0A128A11702678
:101890006730B9001130BA00BC267B267B30B90016
:1018A0001130BA00BC2688260A128A157C08033932
:1018B000A000A0182010A00855300319642C013096
:1018C00020025B30031D61300A128A11A0260A1221
:1018D0008A1188240A128A15A1000F302106031DDF
:1018E000742C0A128A11F12914302106031D7E2C52
:1018F000A00A033020020319A0005B2C153021063A
:10190000031D892CA003FF30200202300319A00020
:101910005B2C0E302106031D672CA030840008309C
:101920000A128A1122242008FC0083160313B60031
:1019300083120313A0308400083044240A128A1151
:10194000AF280A128A1170268F30B9001130BA0000
:10195000BC267B26A430B9001130BA00BC26690829
:101960006F240F39A0000A128A115530A0260A30C0
:1019700020020030031806302007D0260A128A11F0
:1019800088240A128A15A1000F302106031DCB2CD2
:101990000A128A11F12914302106031DD52C0F30AB
:1019A00020060319BE2CA00AB32C15302106031DF6
:1019B000DE2CA0080319BE2CA003B32C0E30210688
:1019C000031DBE2C20080A128A117B24E900AF28CF
:1019D0000A128A117026B930B9001130BA00BC263B
:1019E000A0010A128A117B260A128A152008A1007A
:1019F000A10AA10BFF2CCE30B9001130562DA10B3E
:101A0000052DD830B9001130562DA10B0B2DE1302A
:101A1000B9001130562DA10B112DEA30B90011304B
:101A2000562DA10B172DF430B9001130562DA10BF6
:101A30001D2DFE30B9001130562DA10B232D08307D
:101A4000B9001230562DA10B292D1230B9001230D9
:101A5000562DA10B2F2D1C30B9001230562DA10B85
:101A6000352D2630B9001230562DA10B3B2D3030CC
:101A7000B9001230562DA10B412D3A30B900123069
:101A8000562DA10B472D4430B9001230562DA10B15
:101A90004D2D5530B9001230562DA10B532D61300C
:101AA000B9001230562D7030B9001230BA000A1247
:101AB0008A11BC260A128A1188240A128A15A100EA
:101AC0000F302106031D672D0A128A11F1291430E7
:101AD0002106031D712DA00A103020060319A00055
:101AE000F12C15302106031D7C2DA003FF302006AC
:101AF0000F300319A000F12C0E302106031D5A2DC2
:101B000020080A128A11E32577250A128A155A2D10
:101B10000A128A1170267F30B9001230BA00BC2632
:101B20007B268D30B9001230BA00BC268826A00171
:101B3000B318A00A5630201C5E300A128A11A02663
:101B40000A128A1188240A128A15A1000F30210670
:101B5000031DAD2D0A128A11F12914302106031933
:101B6000B52D15302106031DB82D0130A0069A2D84
:101B70000E302106031DA02DB3102018B3140A1235
:041B80008A11AF28EF
:10200000203454346834653420344E3469346334B5
:102010006534203443346F346E34743472346F3426
:102020006C3400342034203466346F3472342034FD
:1020300046345034473441342034743475346E346B
:102040006534723400342034203420342034203479
:102050006234793420346834693472346F346B34C8
:1020600075346E3400342034203476346534723460
:102070002E34323430343134353430343534313434
:1020800036345F347234653400347E344D34613418
:1020900069346E3420346D3465346E3475340034F4
:1020A000283431342934503472346534733465340F
:1020B00074340034283432342934503472346F3458
:1020C0006734723461346D34203465346434693477
:1020D0007434003428343334293453347434613440
:1020E000743469346F346E3420346E3461346D343A
:1020F00065342034653464346934743400342834ED
:1021000034342934413472346534613420345234E7
:102110006534713475346534733474340034283460
:1021200035342934413472346534613420344334D5
:102130007534733474346F346D3469347A3465347F
:10214000003428343634293453342F345034443452
:102150004934463420347234613474346534003484
:102160002834373429344F3475347434703475342A
:10217000743420344C346534763465346C34003433
:10218000283438342934533465346E34643420347C
:1021900049345234203463346F3464346534003449
:1021A0002834393429345334703465346334693411
:1021B00061346C3420346D346F34643465340034ED
:1021C0007E3450347234653473346534743400347E
:1021D00050343134323433343434353436343734A3
:1021E0003834203449346E346934743453345434BC
:1021F00000347E34503472346F3467347234613456
:102200006D342034653464346934743400345034AB
:10221000313432343334343435343634373438347A
:10222000203443346C346534613472342034533494
:1022300061347634653400347E34503472346F3413
:102240006734723461346D342034733474346134DF
:1022500074347534733400347E34533474346134DC
:10226000743469346F346E3420346E3461346D34B8
:102270006534203465346434693474340034503443
:10228000313432343334343435343634373438340A
:1022900000347E3441347234653461342034523435
:1022A00065347134753465347334743400347E3479
:1022B00041347234653461342034433475347334BA
:1022C00074346F346D3469347A34653400347E3458
:1022D00053342F3450344434493446342034733426
:1022E00061346D3470346C3465342034723461344C
:1022F0007434653400342034343438346B34483426
:102300007A342034393436346B3448347A342034D7
:102310003134393432346B3448347A3400347E34D6
:102320004F347534743470347534743420344C3410
:102330006534763465346C342034283430342D34AC
:1023400031343534293400342034303433342034BB
:1023500028345334743461346E34643461347234E8
:1023600064342034693473342034303433342934C1
:1023700000347E34533465346E346434203449344C
:102380005234203463346F34643465342034283458
:1023900030342D3431343534293400342034203471
:1023A0003034303420345B343C343C345D340034DD
:1023B000203420343034313420345B343C345D34C8
:1023C0000034203420343034323420345B343E3412
:1023D0005D340034203420343034333420345B34E2
:1023E0003E343E345D3400342034203430343434D0
:1023F00020345B34503431345D34003420342034A4
:102400003034353420345B34503432345D3400346D
:10241000203420343034363420345B345034333478
:102420005D340034203420343034373420345B348D
:10243000503434345D340034203420343034383473
:1024400020345B34503435345D340034203420344F
:102450003034393420345B34503436345D34003415
:10246000203420343134303420345B345034373429
:102470005D340034203420343134313420345B3442
:10248000503438345D340034203420343134323424
:1024900020345B34623461346E34643477346934AC
:1024A0006434743468345D3400342034203431347E
:1024B000333420345B346D346F34643465345D34CC
:1024C0000034203420343134343420345B345034FC
:1024D000723465347334653474342D345D340034AF
:1024E000203420343134353420345B345034723469
:1024F00065347334653474342B345D3400347E3485
:102500005334703465346334693461346C3420344A
:102510006D346F34643465340034203420344534F1
:102520006E34613462346C34653420342034443485
:1025300069347334613462346C3465340034123479
:1025400034340034FF34123434340134FE34123461
:1025500034340234FD34123434340334FC34123451
:1025600034340434FB34123434340534FA34123441
:1025700034340634F934123434340734F834123431
:1025800034340834F734123434340934F634123421
:1025900034340A34F534123434340B34F434123411
:1025A00034340C34F334123434340D34F234123401
:1025B00034340E34F134123434340F34F0340F34F4
:1025C0000E340C3408340C340E340F3480341E3482
:1025D0000E340634023406340E341E348034113482
:1025E0000A348034153480340A3411348034803411
:1025F000803404340E340434803480348034003425
:10260000203413344D3413347B341334BC3413343A
:10261000FB3413345F341434CA341434FE341434A9
:102620004A3415349C341534E934153429341634BD
:1026300086341634CA3416342F34173466341734BB
:10264000303431342034CE34AF34B634B234C434C0
:10265000DE34B33400343834303434344134493423
:1026600052342D344734273400343834323435343E
:102670004E344F3452345434483420345734413477
:102680005634453400343834353432344E344834DA
:102690004B34203446344D34FF343034323420341B
:1026A000C434B334CE34B8342D34313400343734F8
:1026B0003634313446344D3420344934573441347F
:1026C00054344534003438343034303441344634B2
:1026D00042340034383432343834413446344D34A2
:1026E00000343834333431344E3448344B342034AD
:1026F00046344D34FF34303433342034C434B334AE
:10270000CE34B8342D3432340034373437343134A5
:102710004434613474346534203466346D340034A8
:10272000383430343434523468347934743468345E
:102730006D342034533474346134743469346F34F8
:102740006E340034383431343834463475346B34B4
:1027500075347334683469346D34613420344634EC
:102760004D3400343834323435344E3448344B34FC
:10277000203446344D34FF34303434342034B634CD
:10278000DD34C434B3342D3431340034373436348A
:10279000343452344134443449344F342034423494
:1027A00045345234523459340034373438343834A0
:1027B00048346F3473346F342034443461346934B2
:1027C000673461346B347534003438343034333426
:1027D0004E3448344B34203446344D34003438348D
:1027E0003634333446344D342034473455344E3443
:1027F0004D344134FF34303435342034B634DD3494
:10280000C434B3342D3432340034373436343134B4
:1028100049346E3474346534723446344D34003483
:1028200037343834303462346134793466346D345A
:10283000003437343834363446344D342D3446344D
:1028400055344A3449340034373439343534463415
:102850004D3420344E34413443344B343534003419
:1028600038343034303454344F344B3459344F349A
:10287000203446344D3400343834313433344A341F
:102880002D345734413456344534003438343234DE
:1028900035344E3448344B34203446344D340034CF
:1028A00038343434373446346D34203479346F342A
:1028B0006B346F34683461346D346134FF343034D8
:1028C00036342034B634DD34C434B3342D343334A8
:1028D000003437343634313449346E34743465342A
:1028E000723446344D340034373439343534463458
:1028F0004D3420344E34413443344B343534003479
:1029000038343034303454344F344B3459344F34F9
:10291000203446344D3400343834313433344A347E
:102920002D3457344134563445340034383435343A
:1029300031344E3448344B34203446344D34003432
:1029400039343034353454344234533420345234EE
:102950004134443449344F3400343934313436341A
:10296000423475346E346B346134203468346F34DF
:1029700073346F3400343934333430344E34693482
:10298000703470346F346E34203468346F34733480
:102990006F34FF34303437342034C134AD34B33481
:1029A000CC34DE3400343734393432344B342D34C3
:1029B0004D3449345834003437343934373446349C
:1029C0004D342D344E344134473441344E344F3439
:1029D000003438343334303446344D342D344634B6
:1029E00055344A34493400343834353436344E346E
:1029F00048344B34203446344D34FF34303438348A
:102A00002034C434B334B634B234003437343734B9
:102A100038345A34493450342D3446344D3400342B
:102A200037343834393472346134643469346F344F
:102A30002034433455344234453400343734393447
:102A4000353449346E3474346534723446344D341C
:102A5000003438343034303446344D342034473444
:102A600049344634553400343834303437344634FD
:102A70004D3420346134693463346834693400344B
:102A80003834323435344E3448344B3420344634C0
:102A90004D34FF34303439342034CE34B834D83463
:102AA000B834003437343634313446344D3420347D
:102AB000463455344B345534493400343734373484
:102AC000353446344D342D344E344934493447344A
:102AD000413454344134003437343934303446349A
:102AE0004D34203450344F3452345434003438345C
:102AF00030343534483445344C344C344F3420343D
:102B0000463449345634453400343834323432345F
:102B10004E3448344B34203446344D340034383449
:102B20003234373446344D34203454344F345934ED
:102B300041344D344134FF34313430342034B734EF
:102B4000DD34B7342D343134003437343634353451
:102B500046344D34203443344F3443344F344C34B2
:102B60004F34003438343034323446344D34383411
:102B700030343234003438343534313446344D3422
:102B800020344F34533441344B34413400343834DE
:102B9000383431344E3448344B34203446344D3498
:102BA0000034383439343434E0342D34533454342C
:102BB0004134543449344F344E3400343834393489
:102BC00039344B34693473347334203446344D34DF
:102BD000FF34313431342034B734DD34B7342D345C
:102BE0003234003437343734303465342D34723471
:102BF0006134643469346F340034383430343234FE
:102C000046344D343834303432340034383435348A
:102C1000313446344D3420344F34533441344B3402
:102C2000413400343834373434344E3448344B343F
:102C3000203446344D340034383439343434E034BC
:102C40002D34533454344134543449344F344E3495
:102C5000FF34313432342034C134AD34B334BA3477
:102C6000DE34B834003437343634383446344D34F6
:102C700020344F344B344134593441344D34413491
:102C8000003437343734343456342D3461346934B5
:102C900072340034373438343234483446344D34A6
:102CA000003437343934323446344D3459340034F6
:102CB0003834383433344E3448344B34203446348A
:102CC0004D3400343734373436344B34693473344C
:102CD0007334203446344D34003437343834363489
:102CE00046344D3420344B34413447344134573426
:102CF0004134003437343934373446344D34203499
:102D00004534483449344D344534FF343134333458
:102D10002034BC34BA34B834003437343834363420
:102D200046344D3420344B344134473441345734E5
:102D30004134003437343934373446344D34203458
:102D40004534483449344D34453400343834303413
:102D5000373446344D34203454344F344B345534A6
:102D60005334483449344D344134003438343134E8
:102D70003634483469342D3453346934783400346B
:102D80003834373437344E3448344B3420344634B6
:102D90004D34FF34313434342034B734AD34B334AB
:102DA000BC34AD34B3342D3431340034373436349C
:102DB00031344C346F3476346534203446344D34F9
:102DC000003437343734343446344D344B340034E3
:102DD00037343734393446344D345334003437348F
:102DE00038343734633472346F347334733420348A
:102DF00066346D34003437343934353446344D3428
:102E000020344E34613467346134733461346B344C
:102E10006934003438343034373446344D34203457
:102E2000463455344B3455344F344B3441340034EC
:102E30003834343438344E3448344B342034463407
:102E40004D340034383438343034413469347234D9
:102E5000203452346134643469346F34FF34313493
:102E600035342034B734AD34B334BC34AD34B3343A
:102E70002D343234003437343734343446344D341E
:102E80004B34003437343934383446344D342034FC
:102E90006B34613467346F347334683469346D343F
:102EA000613400343834333432344A344F34593492
:102EB000203446344D3400343834353436344E34CE
:102EC00048344B34203446344D34FF3431343634B6
:102ED0002034B534B734C534DC34003438343734B6
:102EE000333466346D3420346F346B3469346E346B
:102EF00061347734613400343834383431344E340A
:102F000048344B34203446344D340034383439346A
:0A2F10003134413446344E34FF34AE
:02400E00E42F9D
:02401000FF3F70
:1042000037003600310033003100300049006E00C5
:1042100074006500720046004D0020002000200060
:10422000200020002000200020002000200020008E
:10423000200020003700380030003300310030000B
:1042400062006100790066006D00200020002000FF
:10425000200020002000200020002000200020005E
:1042600020002000200020003700380036003300F6
:104270003100300046004D002D00460055004A0038
:104280004900200020002000200020002000200005
:1042900020002000200020002000200037003900EE
:1042A000350033003100300046004D0020004E0044
:1042B000410043004B00350020002000200020007A
:1042C00020002000200020002000200020002000EE
:1042D00038003000300033003100300054004F000F
:1042E0004B0059004F00200046004D0020002000E8
:1042F00020002000200020002000200020002000BE
:10430000200020003800310033003300310030003D
:104310004A002D00570041005600450020002000B3
:10432000200020002000200020002000200020008D
:10433000200020002000200038003200350033002B
:10434000310030004E0048004B00200046004D0078
:10435000200020002000200020002000200020005D
:104360002000200020002000200020003800340021
:10437000370033003100300046006D002000790026
:104380006F006B006F00680061006D00610020002D
:10439000200020002000200020002000200020001D
:1043A000370036003100330031003000500031005A
:1043B00020002000200020002000200020002000FD
:0E43C00020002000200020002000200000002F
:00000001FF
